:100000000C940B020C9433020C9433020C943302C4
:100010000C9433020C9433020C9433020C9433028C
:100020000C9433020C9433020C9433020C94A616F5
:100030000C9433020C9433020C9433020C9433026C
:100040000C94C4170C9433020C9433020C943302B6
:100050000C9433020C9433020C9433020C9433024C
:100060000C9433020C943302526573756D65005124
:100070007569740068006F000808FC848884A2D148
:100080000A040808003C4299A566180053696E6787
:100090006C6520706C617965722067616D65004DDB
:1000A000756C7469706C617965722067616D65004B
:1000B0004F7074696F6E73008C009F00B000506FBA
:1000C000636B657420456D70697265730003053F4D
:1000D000213F1208120A100A0E1C0E0C1E0C141AD4
:1000E00014161F161E131E1E1B1E1E1F1E3F213F11
:1000F0003A2F3A173D173F213F181F02040A041FE9
:100100000E04040E1F0A1F0A0E0E1F04110E2E25C8
:100110002E2F2A2E262929021F02081F08150E0439
:10012000040E150E15151B151B040604040C040003
:1001300000000017000300031F0A1F16371A1904D6
:10014000130A153A000300000E11110E000A040AEA
:10015000040E040030000404040010001804031FFF
:10016000111F121F101D151711151F07041F17153A
:100170001D1F151D01011F1F151F17151F000A0048
:10018000003200040A110A0A0A110A040115020EBB
:1001900011171E051E1F150A0E110A1F110E1F151D
:1001A000111F05010E111D1F041F111F1108100F33
:1001B0001F041B1F10101F061F1E040F0E110E1F01
:1001C00009060E112E1F051A121509011F011F1015
:1001D0001F0F180F1F0C1F1B041B031C03191513E3
:1001E000001F11030418111F00020102202020002B
:1001F00001020C121E1F120C0C12120C121F0C1AF0
:1002000014041E05242A1E1F021C141D1020201D6C
:100210001F0814111F101E041E1E021C0C120C3E7F
:100220000A040C123E1E040214160A020F120E10CB
:100230001E0E100E1E081E120C1226281E322A2612
:10024000041E21001F00211E040102013F213F0A5C
:100250004E6F2053442063617264206F720A6E6F88
:10026000204C4F414445522E4845580A0A153A45FC
:10027000786974001D20466C617368696E670A2096
:10028000206C6F616465722E2E2E0A0A444F4E2731
:1002900054205455524E204F464621000A0A153A22
:1002A00049676E6F7265006D560A0A504C4541539E
:1002B00045205455524E204F464620004C4F572063
:1002C00042415454455259212000175344001613FB
:1002D0007800161314001510200015201000540A81
:1002E00003E181867F3E186D830F0F0E01838660C8
:1002F00033186DC3198F1803C38E6033186DE33044
:10030000CF1803C39E603630CDE360CF3006C79E62
:100310007E3E30CDB360CF300CC6F6603330D9B6F8
:1003200060CF33CFCCF66061B0DB1E60CF30D86CCD
:10033000E6C061B0DB1E618F19986CC6C063B19BCB
:100340000E330F0FB078C6FF7E1F1B061E0F050071
:10035000893008023802497868140000F6E8DBCFDB
:10036000C3B8AEA49B928A827B746E68625C57525B
:100370004E4945413E3A3734312E2C292725232139
:100380001F1D1C1A1917161514131211100F0E0D1C
:100390000C0B0A0908070645006801000005006803
:1003A00001380100000500380168010000B503B103
:1003B000030101FF030101F7030000000700020130
:1003C0000000030406000000000000000001020419
:1003D00008102040800102040810200102040810C7
:1003E00020040404040404040402020202020203BE
:1003F000030303030300000000230026002900007C
:10040000000000250028002B000000000024002729
:10041000002A00007B0211241FBECFEFD8E0DEBF10
:10042000CDBF11E0A0E0B1E0E4EFFAE302C0059037
:100430000D92A437B107D9F724E0A4E7B1E001C0D9
:100440001D92AE30B207E1F712E0CBE0D2E004C07B
:100450002197FE010E94231CCA30D107C9F70E94D0
:1004600035020C94781D0C9400000E9475020E94C5
:100470007A06FDCFEF92FF920F931F93CF93DF93F6
:100480007C01C0E0D0E000E010E0F701828190E064
:100490000817190768F4808191818C0F9D1F0097C0
:1004A00011F00E9404030F5F1F4FCE5DDD4FEDCFB3
:1004B00084E791E00E94A90F8823D1F366E08EE7DC
:1004C00091E00E948B088823E1F242E064E770E04B
:1004D00084E791E00E946410813099F6DF91CF911A
:1004E0001F910F91FF90EF9008950E94651884E787
:1004F00091E00C94AA131092C5011092C40189E6F0
:1005000091E09093C3018093C2010895EF92FF920E
:100510000F931F93CF93DF93CDB7DEB727970FB617
:10052000F894DEBF0FBECDBF7C010E942004F7010E
:10053000E85EFD4F80819181019769F461E082EC72
:1005400091E00E948A0908E024E548E260E082EC3C
:1005500091E00E94CA0900E022E040E068E770E014
:10056000CE0101960E94720384EEE81A8DEFF80A1C
:10057000C7010E94B506182FC7010E94B206412F7D
:10058000682FCE0101960E94BF03CE0101960E9402
:100590007D0327960FB6F894DEBF0FBECDBFDF9167
:1005A000CF911F910F91FF90EF9008950F931F939C
:1005B000CF93DF93EC018A010E94C30389E091E0AD
:1005C00099838883FE01E85EFD4F11821082329686
:1005D00011830083B801CE01845E9D4F0E948C067A
:1005E000FE01E05EFD4F10823196108220E130E086
:1005F00040E150E061E070E0CE014896DF91CF919C
:100600001F910F910C946705CF93DF93EC010E942B
:100610001A08CE010E940904E881F9810190F08155
:10062000E02DCE01DF91CF9109949F92AF92BF92BE
:10063000CF92DF92EF92FF920F931F93CF93DF93AE
:10064000EC0168966C0128EEC21A2DEFD20A8C01DB
:10065000045E1D4FCE010E944105882389F1CE0121
:100660000E94440581112CC0CE010E944A055C0104
:10067000CE010E944E057C01C8010E94B806982E4A
:10068000C8010E94C00695012919310937FF03C02E
:100690003195219531092032310594F49701281BB9
:1006A0003109C90137FF03C0919581959109809760
:1006B0003CF461E0CE010E94470582E090E006C074
:1006C0006096CC15DD0531F680E090E0DF91CF91AA
:1006D0001F910F91FF90EF90DF90CF90BF90AF9060
:1006E0009F9008950F93FC0171836083428323835D
:1006F0000483158216820F9108950F931F93CF9351
:10070000DF93EC0140E06B8182EC91E00E948E0966
:100710008091FB019091FC01009729F12A816D8164
:10072000222329F070E00E944B048C0101C0062FA7
:100730009A818E81992341F0682F70E08091FB01AE
:100740009091FC010E9453042881398121153105C3
:1007500051F0482F602F82EC91E0DF91CF911F91F3
:100760000F910C94950BDF91CF911F910F910895EC
:10077000FC01849108950196FC0184910895FC0187
:10078000658346830895AF92BF92CF92DF92EF9236
:10079000FF920F931F93CF93DF93EC016B018FE0D8
:1007A00091E0998388837E0188E0E80EF11C80E166
:1007B000F70111928A95E9F78E01085E1F4F5E01DD
:1007C000F8EEAF1AFDEFBF0A60E070E0C8010E94CA
:1007D0005205005F1F4F0A151B05B1F7C114D10464
:1007E00031F040E150E0B601C7010E94691D43E0CD
:1007F00050E06CE271E0CE010296DF91CF911F9143
:100800000F91FF90EF90DF90CF90BF90AF900C943E
:10081000621D0F931F93CF93DF938C01085E1F4FD0
:10082000EC01C85EDD4FC8010E949F05005F1F4FAD
:100830000C171D07C1F7DF91CF911F910F910895FC
:100840000F931F93CF93DF938C01085E1F4FEC0132
:10085000C85EDD4FC8010E94C905005F1F4F0C171D
:100860001D07C1F7DF91CF911F910F910895FC01F2
:100870001082128211821482138215820895FC0163
:1008800081819281860F971F0895FC018381948155
:10089000860F971F0895FC01818192819B01281B7F
:1008A000390BC9010895FC01838194819B01281BA8
:1008B000390BC90108950F931F93CF93DF93EC0178
:1008C0008B01CB010E94C806811109C040E06CEF8A
:1008D000C801DF91CF911F910F910C9494068981EB
:1008E0009A818430910594F304979A838983DF91E8
:1008F000CF911F910F9108950F931F93CF93DF9383
:10090000EC018B01CB010E94C806811109C040E0B7
:1009100064E0C801DF91CF911F910F910C94940670
:1009200089819A81811522E092078CF704969A8337
:100930008983DF91CF911F910F9108950F931F939A
:10094000CF93DF93EC018B01CB010E94CF06811185
:1009500009C04CEF60E0C801DF91CF911F910F916A
:100960000C9494068B819C811816190694F70497B1
:100970009C838B83DF91CF911F910F9108950F93EB
:100980001F93CF93DF93EC018B01CB010E94CF0625
:10099000811109C044E060E0C801DF91CF911F914F
:1009A0000F910C9494068B819C81811522E0920713
:1009B0008CF704969C838B83DF91CF911F910F91CD
:1009C0000895FC0180810895FC0111821082128239
:1009D000138215821482178216820895FC0181E029
:1009E0008283758364835783468308950895909323
:1009F000FE018093FD010895DF92EF92FF920F9325
:100A00001F93CF93DF93FC012381222391F18B016C
:100A10007C01CB010E94B803C82FC8010E94BB0310
:100A2000082F8091FD019091FE01009711F1D0E017
:100A3000F701648175816C1B7D0B0E944B04D82EDD
:100A400010E0F70166817781601B710B8091FD01D9
:100A50009091FE010E945304000F111F9E01220F6E
:100A6000331F52E0E52E482F6D2D82EC91E00E945D
:100A7000FF0ADF91CF911F910F91FF90EF90DF90D0
:100A80000895FC0182810895FC0183810895FC0191
:100A900063830895FC01848195810895FC0186811A
:100AA000978108950F931F93CF93DF93EC018B01F0
:100AB0000E94E404198708871B861A861D861C86F7
:100AC0001F861E86DF91CF911F910F910895EF929F
:100AD000FF920F931F93CF93DF9300D01F92CDB758
:100AE000DEB77C018B01BA01A9010E94EE04F70177
:100AF000118700878091020190910301A091040168
:100B000089839A83AB83FE01E00FF11F818190E01E
:100B1000F701918380830F900F900F90DF91CF9119
:100B20001F910F91FF90EF900895FC0175876487E6
:100B30005787468781E090E0938782870895CF9317
:100B4000DF93EC010E94F6048A859B850197F1F4FE
:100B50008C819D812C853D858217930710F4019629
:100B600004C02817390718F401979D838C838E8160
:100B70009F812E853F858217930710F4019604C04C
:100B80002817390718F401979F838E83DF91CF913F
:100B90000895CF92DF92EF92FF920F931F93CF931E
:100BA000DF93CDB7DEB72D970FB6F894DEBF0FBE3B
:100BB000CDBFFC012085318523303105BCF57C019A
:100BC0001986188682E890E09B878A871D861C8696
:100BD000220F331FE1E0F0E0EC0FFD1FE20FF31FE7
:100BE000C780D08400E021E041E0B601CE0101964B
:100BF0000E947203F7010681C6010E94BB0386951D
:100C0000081BF7011481C6010E94B8038695612F65
:100C1000681B402FCE0101960E94BF03CE010196B2
:100C20000E947D03B601C7010E94FC042D960FB6F9
:100C3000F894DEBF0FBECDBFDF91CF911F910F9112
:100C4000FF90EF90DF90CF900895CF92DF92EF92D8
:100C5000FF920F931F93CF93DF93CDB7DEB7C753A8
:100C6000D2400FB6F894DEBF0FBECDBF8E010D5D32
:100C70001D4F8AE0F80111928A95E9F7B80184E7DF
:100C800091E00E9405147E01F3EDEF1AFDEFFF0ADB
:100C9000C7010E943704A701B801CE0101966C017B
:100CA0000E94D602005F1F4F85E0F80111928A95DD
:100CB000E9F781E0F8018283D182C082F482E38285
:100CC000F092FC01E092FB01C7010E94F704C80109
:100CD0000E943A02C95CDD4F0FB6F894DEBF0FBE2A
:100CE000CDBFDF91CF911F910F91FF90EF90DF90DB
:100CF000CF9008956EEB70E084E791E00E942D1391
:100D000043E068EB70E084E791E00E946410811199
:100D100002C00C9425060895FC0188E2808386E1D8
:100D20008183738362830895FC019081262F062EB0
:100D3000000C330B290F311D97FD3A9529323105EF
:100D400010F4960F90838181242F042E000C330B16
:100D5000280F311D87FD3A952731310510F4840F96
:100D600081830895FC0180810895FC0181810895AB
:100D7000FC01608170E0828193810E943F040895AC
:100D8000FC01618170E0828193810E944504089595
:100D9000FC0181E09081983209F080E0089521E023
:100DA000FC018181863109F020E0822F0895DC0169
:100DB000A85EBD4F2D913C911197FC01E05EFD4F67
:100DC0002230310539F48081853020F081E090E0D7
:100DD0008D939C9310820895AF92BF92CF92DF9231
:100DE000FF920F931F93CF93DF93EC016C0188EE7A
:100DF000C81A8DEFD80AF60180819181029701F51A
:100E00008E01085E1F4F5E01F4EEAF1AFDEFBF0AC0
:100E1000C8010E944405882371F0C5010E94B806EC
:100E2000F82EC5010E94C006482F50E06F2D70E0DB
:100E3000C8010E949505005F1F4F0C151D0541F765
:100E4000CF5DDD4F1882DF91CF911F910F91FF9001
:100E5000DF90CF90BF90AF900895EF92FF920F93E5
:100E60001F93CF93DF938C010F5D1D4FF8012081FD
:100E70002F5F20832A30C8F07C01F8EEEF1AFDEFD7
:100E8000FF0AF701208131812230310561F4EC0144
:100E9000689660E0CE010E9447056096CE15DF059A
:100EA000C1F719821882F8011082DF91CF911F914A
:100EB0000F91FF90EF900895CF93DF93EC01C85E00
:100EC000DD4F288139812115310521F0223031058E
:100ED00031F00DC00E9415039983888308C0FC017E
:100EE000E05EFD4F80818F3F11F08F5F8083DF9147
:100EF000CF910895DB01AA0FBB1FAA0FBB1FA75BF1
:100F0000BE4FED91FC91119712962D913C91139744
:100F1000A90141705527309719F44115510589F001
:100F200035952795452B51F0DC01A20FB31F4D914C
:100F30005C91E40FF51F0190F081E02D820F931F6B
:100F400009940895EF92FF920F931F93CF93DF932D
:100F50008C01EB017C0186EEE81A8DEFF80AD701CF
:100F60008D919C910E94E104811135C0DE01AA0F90
:100F7000BB1FAA0FBB1FA35DBE4FED91FC91119744
:100F800012968D919C9113979C0121703327309775
:100F900019F421153105F9F095958795232B61F00A
:100FA000E701A881B981A80FB91F2D913C91E20FEB
:100FB000F31F0190F081E02DB801645E7D4FD701F1
:100FC0002D913C91820F931FDF91CF911F910F9133
:100FD000FF90EF900994DF91CF911F910F91FF90B7
:100FE000EF900895DB01AA0FBB1FAA0FBB1FAF5ED6
:100FF000BE4FED91FC91119712962D913C91139754
:10100000A90141705527309719F44115510589F010
:1010100035952795452B51F0DC01A20FB31F4D915B
:101020005C91E40FF51F0190F081E02D820F931F7A
:10103000099408950F931F93CF93DF938C01C0E021
:10104000D0E06C2F8EE791E00E94AC08882349F035
:10105000BE01C8010E947A07BE01C8010E94A20712
:101060000BC06C2F8EE791E00E948B08882321F043
:10107000BE01C8010E94F2072196C730D10509F7C9
:10108000DF91CF911F910F910895FC0188E080833B
:1010900089E0818387E0828386E0838384E08483A0
:1010A00082E0858381E186830895FF920F931F93E9
:1010B000CF93DF93EC018C01095F1F4FFF24FA945B
:1010C00062E088810E94451988810E94B0192F81B1
:1010D000892B19F42F5F2F8307C0222349F02F3F5C
:1010E00011F41F8201C0FF8260E088810E944519CF
:1010F0002196C017D10721F7DF91CF911F910F9152
:10110000FF900895FC01E60FF11D81E09781913079
:1011100009F080E00895FC01E60FF11D81E0978160
:101120009F3F09F080E00895262F30E0FC01E20F98
:10113000F31F423030F49781915081E09E3F58F088
:1011400009C087818F3F31F0642F0E94A31B81E08B
:10115000913009F080E00895860F911DFC01878190
:101160008F3F09F480E008958EBD0DB407FEFDCFDA
:101170008EB50895DC01643508F057C0403308F09F
:1011800054C090969C919097E42FE595E595E59550
:10119000262F062E000C330B542F57709230A1F4DB
:1011A000D90184E5E802A00DB11D1124A150BE4F64
:1011B0008C9190E0052E02C0959587950A94E2F7F0
:1011C0008095982F91700CC0933051F41C968C919F
:1011D0006427062E000C770B682760FF03C014C03D
:1011E000911112C084E5E802200D311D1124F9018E
:1011F000E150FE4F81E090E001C0880F5A95EAF778
:1012000080959081892310C084E5E802200D311D6E
:101210001124F901E150FE4F81E090E001C0880FF8
:101220005A95EAF79081892B808308951F93CF9375
:10123000DF93EC01162FF89460E08F850E948119EE
:10124000888918161CF460E00E948119812F0E9481
:10125000B408888918161CF461E00E9481197894FA
:10126000DF91CF911F91089528EF31E0EFEFF1E08A
:10127000DF01A9011D9241505040E1F7DC011996B0
:101280001C9219971A961C920895CF92DF92EF92B2
:10129000FF920F931F93CF93DF93EC018C858F5FA9
:1012A0008C878FEFE82E81E0F82E10E0612F6064CC
:1012B000CE010E94160960E8CE010E94160961E085
:1012C0008F850E948119888918161CF460E00E949D
:1012D0008119670104E5F60181916F010E94B4084C
:1012E0000150C9F7888918161CF461E00E94811921
:1012F0001F5FF4E5EF0EF11C1630C1F660E4CE017D
:10130000DF91CF911F910F91FF90EF90DF90CF90E1
:101310000C941609FC0160A361A30895FC0160A36D
:1013200041A30895EF92FF920F931F93CF93DF9302
:101330008C01D62FF42EE22EC0E0CE1544F44F2DB2
:101340004C0F6D2FC8010E94BA08CF5FF6CFDF9116
:10135000CF911F910F91FF90EF900895EF92FF9220
:101360000F931F93CF93DF938C01F62ED42FE22E91
:10137000C0E0CE1544F46F2D6C0F4D2FC8010E94B4
:10138000BA08CF5FF6CFDF91CF911F910F91FF90F9
:10139000EF900895EF92FF920F931F93CF93DF93F7
:1013A0007C01C62F142FD22F0E94AE094FEF400FA1
:1013B000410F2D2F6C2FC7010E94AE09202F412F06
:1013C0006C2FC7010E9492096FEF6D0F6C0F202FD9
:1013D000412FC701DF91CF911F910F91FF90EF90A7
:1013E0000C949209DF92EF92FF920F931F93CF9389
:1013F000DF937C01D62FD22EC42F002E000C110BB0
:10140000040F111D47FD1A958C2F0C2E000C990B03
:101410008017910744F42D2D4C2F6D2FC7010E948A
:10142000AE09CF5FF1CFDF91CF911F910F91FF9068
:10143000EF90DF9008958F929F92AF92BF92CF92DC
:10144000DF92EF92FF920F931F93CF93DF937C0174
:10145000162FD42EC22F81E0C82EC21AB22EB194FC
:10146000BB0CD0E0802F8470A82E802F8270982E25
:10147000802F8870882E0170DC170CF04DC0C7FCDF
:1014800004C0C150B394B394CB0CDF5F8D2F880F91
:101490008F5FC80EAA2071F04D2D4C0F612F6D0F7C
:1014A000C7010E94BA084D2D4D0F6C2F610FC70167
:1014B0000E94BA08992071F04D2D4C1B612F6D0FC1
:1014C000C7010E94BA084D2D4D1B6C2F610FC7013B
:1014D0000E94BA08882071F04D2D4D0F612F6C1BB2
:1014E000C7010E94BA084D2D4C0F612F6D1BC7011B
:1014F0000E94BA08002309F4BFCF4D2D4D1B612F68
:101500006C1BC7010E94BA084D2D4C1B612F6D1B2F
:10151000C7010E94BA08B0CFDF91CF911F910F9100
:10152000FF90EF90DF90CF90BF90AF909F908F9003
:1015300008958F929F92AF92BF92CF92DF92EF92D7
:10154000FF920F931F93CF93DF936C01A62E942EDF
:10155000C22F11E0121BF22EF194FF0C83E0B82E83
:10156000BE0CD1E0802F8170882EE39402708FEF43
:101570008D0F8C17BCF517FD04C0C150F394F39484
:101580001F0D8D2F880F8F5F180F882091F02C2F43
:10159000220F2E0D492D4C1B6D2F6A0DC6010E9486
:1015A00092092B2D492D4D1B6C2F6A0DC6010E94EF
:1015B0009209011104C0DF5FB394B394D8CF2C2FEC
:1015C000220F2E0D492D4C1B6A2D6D1BC6010E944A
:1015D00092092B2D492D4D1B6A2D6C1BC6010E94B3
:1015E0009209E9CFDF91CF911F910F91FF90EF907A
:1015F000DF90CF90BF90AF909F908F9008959F9273
:10160000AF92BF92CF92DF92EF92FF920F931F9310
:10161000CF93DF936C01C62FD42FB22EAE2CAA0C21
:10162000922E9A18FE2CF60E292D6F2D0E94AE09CF
:101630001FEF100F1D0F292D412F6F2DC6010E9486
:10164000AE090A19DE0D202F4D2F6C2FC6010E9406
:101650009209CB0D6FEF6C0F202F4D2FC6010E940A
:10166000920901E02E2D4D2F6F2DC6010E941B0AFD
:101670008E2D8095C80F02E02E2D4D2F6C2FC601A8
:101680000E941B0AD12FDE1904E02E2D4D2F6C2F46
:10169000C6010E941B0A08E02E2D4D2F6F2DC6019A
:1016A0000E941B0ADF91CF911F910F91FF90EF9045
:1016B000DF90CF90BF90AF909F900895AF92BF9270
:1016C000CF92DF92EF92FF920F931F93CF93DF930E
:1016D0006C01B62EF42E122FC02FDE2DEE0CAD2E87
:1016E000A60E2E196A2D0E94F209C150CE19FD0EC8
:1016F0006FEF6B0D610F6D1BEC2E01E02D2F4F2D49
:10170000C6010E94990A02E02D2F4F2D6A2DC601B5
:101710000E94990ADF91CF911F910F91FF90EF9056
:10172000DF90CF90BF90AF9008952F923F925F923D
:101730006F927F928F929F92AF92BF92CF92DF92E1
:10174000EF92FF920F931F93CF93DF93EC01F90178
:10175000E4903196849164350CF019C10E2C000C84
:10176000FF08062F062E000C110BF701E00FF11FEA
:101770001E161F060CF00BC140330CF008C1A82F39
:10178000C42E042E000CDD085601A80EB11C87FDE6
:10179000BA941A141B040CF0FAC02E5F3F4F570185
:1017A00097E0A90EB11CB7FE04C05701BEE0AB0E16
:1017B000B11CB3E0B594A794BA95E1F747FF0AC00E
:1017C000A42FA80FAC9CC001AD9C900D1124281B28
:1017D000390B40E08A2F0A2E000C990B840F911DC3
:1017E00047FD9A95C19714F0A0E3A41BF8A067FDEC
:1017F00060E0E535F10514F0E4E5F0E09E2FCC85DE
:10180000C427C62E062E000CDD08F601E01BF10BE6
:101810008F014F01F7E08F229924E0E8F0E002C049
:10182000F595E7958A94E2F77E2F17FF02C0095FCE
:101830001F4FF3E015950795FA95E1F7200F311F3B
:10184000542F577081E001C0880F5A95EAF74595EB
:1018500045954595F601B4E54B02E00DF11D1124C7
:10186000AF0141505E4FD0E02A2EAA0F3308EE247C
:10187000E394BB24ED2FF0E0E215F3050CF087C0F4
:10188000F9015490F1E0FF121AC0962E8A01E72F59
:101890006901991608F072C08E2E852021F0D801BA
:1018A0008C90882A8C92E69531F4BFEFCB1ADB0A34
:1018B000F6015490E0E893940F5F1F4FEACFF110C8
:1018C0001CC0782E7094962E8A01E72F6901991614
:1018D00008F054C08E2E852021F0D8018C908720EE
:1018E0008C92E69531F4BFEFCB1ADB0AF6015490E7
:1018F000E0E893940F5F1F4FEACFF3E0FF1629F063
:10190000962E8A01E72F690137C0682E6094862ED3
:101910008A01972E69018916D8F4E92DE52159F03D
:10192000D801EC917C2E782470FE02C0E82B02C016
:10193000E621D801EC93969439F4BFEFCB1ADB0A79
:10194000F6015490E0E89E2E83940F5F1F4FE3CF83
:10195000CE2514C08E2E852021F0D8018C908826AB
:101960008C92E69531F4BFEFCB1ADB0AF601549066
:10197000E0E893940F5F1F4F991660F3880F19F4F6
:101980004C5A5F4F81E0DF5F2A0D3B1D73CFDF9123
:10199000CF911F910F91FF90EF90DF90CF90BF906C
:1019A000AF909F908F907F906F905F903F902F901F
:1019B0000895DC01FB0184918F5F14968C9314973A
:1019C0003196E491EF5F1596EC9315976E5F7F4F1C
:1019D0005F967C936E935E970895EF920F93CF93EB
:1019E000DF93EC014E876D872F87E98A088B81E0B2
:1019F000888788A319A28F836DEC70E0CE010E94C6
:101A0000D90C0E94601B81E00E94761B85E00E9439
:101A1000841B8CE00E947F1B61E08E850E9445192B
:101A200061E08D850E94451961E08F850E9445190E
:101A3000898918161CF461E00E94451988891816D6
:101A40001CF461E00E944519898918166CF460E065
:101A50000E9481196AE070E080E090E00E943F18E7
:101A600061E089890E9481198D85082E000C990BEF
:101A7000FC01EF51FC4FE491F0E0EE0FFF1FE1504D
:101A8000FC4F259134913D8B2C8BFC01E353FC4F93
:101A9000E491EB8F8E85082E000C990BFC01EF5121
:101AA000FC4FE491F0E0EE0FFF1FE150FC4F259159
:101AB00034913B8B2A8BFC01E353FC4FE491EA8F7A
:101AC0008889082E000C990BFC01EF51FC4FE49122
:101AD000F0E0EE0FFF1FE150FC4F259134913F8B5A
:101AE0002E8BFC01E353FC4FE491EC8F8F85082E85
:101AF000000C990BFC01EF51FC4FE491F0E0EE0F6C
:101B0000FF1FE150FC4F25913491398F288FFC0144
:101B1000E353FC4FE491ED8F61E2CE010E94160980
:101B200064E1CE010E9416098B8587FF02C08FE712
:101B30008B876B856068CE010E94160960E2CE013A
:101B40000E9416096CE0CE010E941609CE01DF91B9
:101B5000CF910F91EF900C9445096F927F928F92E5
:101B60009F92AF92BF92CF92DF92EF92FF920F932C
:101B70001F93CF93DF93EC0164350CF084C04033A6
:101B80000CF081C0EC81F0E031970E9FC0010F9FF7
:101B9000900D1124860F911D67FD9A951816190650
:101BA0000CF071C03D81842F042E000C990B039F13
:101BB000800D911D1124181619060CF064C0D02E4A
:101BC000B42EC62E88A0A62E962EE22EF12CEA2D3B
:101BD000EC190E2E000CFF0B8C8190E0E817F90732
:101BE0000CF050C00197E817F90779F0E89E9001D2
:101BF000E99E300DF89E300D1124E20FF31F8E8DFB
:101C00009F8DE80FF91F149101C010E07B2C6B2C05
:101C1000272D2B19022E000C330B8D8190E02817F5
:101C200039076CF510FF11C081E0D81206C0472DAE
:101C30006A2DCE010E94BA081EC00D2D2D2D462DF5
:101C4000692DCE010E94F20916C089A198A18917B9
:101C500091F088A381E0D81206C0472D6A2DCE01ED
:101C60000E94BA0807C00D2D2D2D462D692DCE01DD
:101C70000E94F20988A216956D0C7394C9CF9D0C31
:101C8000A394A5CF88A2DF91CF911F910F91FF90D0
:101C9000EF90DF90CF90BF90AF909F908F907F900C
:101CA0006F9008950F93CF93DF93EC016A3011F496
:101CB00028851EC06D3019F1262F08854A85698553
:101CC0000E94AD0D28853C818985239F800D1124BC
:101CD00089879F81992399F0082E000C990B44E580
:101CE00050E0239F401951091124481759073CF42B
:101CF0009D818A85299F800D11248A87198681E01C
:101D000090E0DF91CF910F9108958F929F92AF92C3
:101D1000BF92CF92DF92EF92FF920F931F93CF93D8
:101D2000DF93EC015C0186E8A80EB11CD5019C9103
:101D3000992309F44DC09C3018F41CE0191B01C014
:101D400010E0FE01EA5AFF4F81E080836E01BEE49D
:101D5000CB0ED11C60E0C6010E948A094E01E3E56A
:101D60008E0E911CD4018C9103E0080F9DE2F92E98
:101D70004F2D481B410F23E0E22E24E560E0C60111
:101D80000E945E0B61E0C6010E948A09F401808115
:101D900003E0080F4F2D481B410F24E560E0C6010A
:101DA0000E94FF0AFE01E95AFF4F84E080833196CA
:101DB000D4018C91181B115D1083CC57DF4F6881C3
:101DC0007981C6010E94161AF501808181508083B5
:101DD000DF91CF911F910F91FF90EF90DF90CF9007
:101DE000BF90AF909F908F900895CF92DF92FF9217
:101DF0000F931F93CF93DF93FC01248D358D232BFD
:101E000009F49FC0EC018C01025B1F4F40E061E0D0
:101E1000C8010E948E09FE01E95AFF4FDE01AE5A49
:101E2000BF4F9C9185E5891B808331961082698D17
:101E3000613009F463C028F0888D653008F074C003
:101E40006FC0CE0185960E944B1581E0FE01EA5AD3
:101E5000FF4F80836DEC70E0C8010E94D90C1D8E8D
:101E60001C8EFE01EC5AFF4F108288EAF82E6E019C
:101E7000FAE0CF0ED11CCE010E94A90F8823D9F31E
:101E80006CEB72E0C8010E94161A6A8D7B8D4AE0E5
:101E900050E0C8010E94C91A67EA72E0C8010E94B6
:101EA000161A6F2D62956F7070E04AE050E0C8011D
:101EB0000E94171B6CE972E0C8010E94161A64E0C8
:101EC000C6010E94820881113CC0FA94F110D3CF60
:101ED00060E0CE010E941E1783B7817F846083BFBC
:101EE00083B7816083BF83B7816083BF889583B7E1
:101EF0008E7F83BF83B78E7F83BFBDCFCF58DF4F29
:101F000088819981AA81BB818F709927AA27BB27D5
:101F10000897A105B10510F467E009C068E707C09C
:101F2000882379F06B5F03C0882359F06FE2C80102
:101F3000DF91CF911F910F91FF90DF90CF900C9484
:101F4000391ADF91CF911F910F91FF90DF90CF90C1
:101F500008958F929F92AF92BF92CF92DF92EF92AD
:101F6000FF920F931F93CF93DF93EC017C0180E8E6
:101F7000E80EF11CF70180809180A280B3800E945E
:101F80000E18861A970AA80AB90A6E01FFE7CF0E43
:101F9000D11CF601808190E0A0E0B0E08E010558F0
:101FA0001F4F88159905AA05BB0550F4F8018081DB
:101FB0009181A281B381892B8A2B8B2B09F040C0A0
:101FC000F80180819181A281B381892B8A2B8B2B8F
:101FD000A9F57E01F5E2EF0EF11CC7010E9448153C
:101FE000C7010E94B415C7010E947916CE010E9454
:101FF000850ECE010E94F50E7E018EE4E80EF11CE6
:10200000C7010E944509FE01EC5AFF4F80818111F2
:1020100003C0C7010E9434090E941A18F8016083A6
:10202000718382839383FE01EB58FF4FC958DF4FC2
:1020300028813981621B730B7183608380E037C014
:102040000E940E18F6012081DC01CB01820F911D48
:10205000A11DB11DF70180839183A283B383FE018B
:10206000EF58FF4F80819181A281B3810196A11D1C
:10207000B11D80839183A283B383F8011082118202
:10208000128213820E941A18FE01E958FF4F6083E2
:10209000718382839383CE010E942217CE010A9618
:1020A0000E945508CE0148960E948B1781E0DF916F
:1020B000CF911F910F91FF90EF90DF90CF90BF9045
:1020C000AF909F908F9008952F923F924F925F9282
:1020D0006F927F928F929F92AF92BF92CF92DF9238
:1020E000EF92FF920F931F93CF93DF93CDB7DEB79D
:1020F00065970FB6F894DEBF0FBECDBF6C016A8B3B
:102100007B8B4B83FC01EC5AFF4F10822FEF2D830A
:102110001C821D8A10E31C8A5C013AE0A30EB11CEC
:102120001C0183E5280E311CBF972F01242F30E0BE
:102130003F832E83C601895A9F4F99878887F396DC
:10214000FB87EA8796012A5A3F4F3F872E870297DF
:10215000998B888B3A973F01C6010E94A90F88236B
:10216000D9F364E0C5010E948208012F110F110B01
:10217000811144C065E0C5010E94820881113EC002
:1021800066E0C5010E948208811138C02C812111AE
:102190004CC044E063E0C5010E949408882331F0FC
:1021A0003C893F5F3C8BC2010E94F61644E061E02F
:1021B000C5010E949408882331F08C8981508C8B52
:1021C000C2010E94F616EC898E2F0E2E000C990B80
:1021D0002E813F818217930731F0E7FF05C03B81D5
:1021E00031503C8B01C01C8AF1018081F4E0F80F72
:1021F0002C89829FF0191124FD8B22C0F101F081FE
:10220000F98364E0C5010E948208882309F48CC028
:10221000C2010E94CA16FC89FD83298121953B8158
:10222000239F302D112432503D8BC8013D89831BE3
:10223000910937FD939502970CF47AC081E08C8365
:102240009D89090F111D97FD1A9517FF02C00F5F99
:102250001F4FF801F595E795FA83E9830981102F5F
:10226000E885F9851082EA85FB85008381E0EE85AB
:10227000FF858083E889F9891082EA88FB88812CB0
:10228000912C2C89022E000C330B3D872C878E81DC
:102290009F818816990609F1EC85FD85E815F905F9
:1022A00079F423E0E885F9852083F1018081F02F1E
:1022B0002C89289FF00D11248F2FEA85FB858083C0
:1022C000F70165917491C3010E94541AFFEF8F1AB0
:1022D0009F0A22E0E20EF11CDACF60E0C3010E9407
:1022E0008A09F10180814981FC89F89F400D112400
:1022F000415024E560E0C3010E94AE0961E0C301E2
:102300000E948A09F101808103E0080F4981FC895C
:10231000F89F400D1124425083E0E82E24E560E050
:10232000C3010E94FF0A18CFC2010E94E01675CFB8
:102330008D8165960FB6F894DEBF0FBECDBFDF91DD
:10234000CF911F910F91FF90EF90DF90CF90BF90B2
:10235000AF909F908F907F906F905F904F903F9045
:102360002F9008950F931F93CF93DF93EC018C016F
:10237000025B1F4FC8010E94340964E772E0C80184
:102380000E94161AC8010E94450983E00E94841B1E
:102390008DE691E0EEEFFFE30995FE01EC5AFF4F69
:1023A00010826FE472E0C8010E94541AC8010E94B2
:1023B00045092A96CE010E94550864E0CE010E948C
:1023C0008208811107C062E370E080E090E00E9423
:1023D0003F18F0CFDF91CF911F910F9108952F9269
:1023E0003F924F925F926F927F928F929F92AF92A5
:1023F000BF92CF92DF92EF92FF920F931F93CF93F2
:10240000DF93CDB7DEB729970FB6F894DEBF0FBEC6
:10241000CDBF3C0120E7620E711CF3012081222315
:1024200009F402C15A011B01998788877A9781E0D4
:102430008083E885F985EB5AFF4F1082E885F9859E
:10244000EC5AFF4F1082E885F985108E8F01025BF0
:102450001F4F61E0C8010E948A09888599858D5ABD
:102460009F4F9D838C83C884D98497E5C90ED11C66
:10247000E884F984E8E5EE0EF11C888599858E5A8A
:102480009F4F9A838983E885F985EF58FF4FFF8333
:10249000EE8388849984FAE08F0E911C48845984D5
:1024A00025E2420E511C888599850E94A90F882338
:1024B000D1F3F1018491882329F0EC81FD81F08131
:1024C000FB8301C01B822EED32E040E060E0C801DA
:1024D0000E94950BA114B10439F04B81445F950122
:1024E00060E0C8010E94950BF60110822CE0F70114
:1024F0002083B101C8010E94161AE981FA81808106
:10250000982F990F890F81958D5AF6018083EC8160
:10251000FD818081982F990F890F8195835DF70147
:102520008083EE81FF81808184FF03C06AED72E0C9
:1025300002C066ED72E0C8010E94541AE981FA8176
:102540008081982F990F890F81958D5AF60180838C
:10255000F70180818F5F8083E885F98582A58823D4
:1025600019F062ED72E002C06EEC72E0C8010E94E8
:10257000541AE981FA818081982F990F890F8195EA
:102580008D5AF6018083F70180818F5F80836AEC2A
:1025900072E0C8010E94541A65E0C4010E948208DA
:1025A000882351F0E885F98562A56F5FC2010E941A
:1025B0000C17C2010E94F61664E0C4010E94820852
:1025C000811113C0F3012081422F50E060E070E0E0
:1025D000EE81FF8180819181A281B381841795076B
:1025E000A607B707A8F02F3F99F08FEFF30180837C
:1025F000088519850B5D1F4F60E0C8010E94E91432
:10260000C8010E94CA1681E0E885F985808F0CC058
:1026100066E0C4010E948208882309F444CF8885BB
:1026200099850E94B21135CF29960FB6F894DEBF76
:102630000FBECDBFDF91CF911F910F91FF90EF9013
:10264000DF90CF90BF90AF909F908F907F906F90D2
:102650005F904F903F902F90089540E050E00C9491
:10266000EF11E0E8F7E72591349181E02130304C1B
:1026700009F080E00895CF93DF93EC010E943113BD
:102680009E01275A3F4FDE01A059BF4F882309F40E
:102690003CC0E6E9F7E78491F9018083E7E9F7E7D1
:1026A000E491EC83E8E9F7E7E491ED83E9E9F7E702
:1026B000859194919F838E83EBE9F7E785919491BF
:1026C00099878887EDE9F7E7E491EBA7EEE9F7E76B
:1026D000E491EAA7EFE9F7E7E491EC93E0EAF7E7A2
:1026E000859194919D8F8C8FE2EAF7E78591949183
:1026F0009F8F8E8FE4EAF7E78591949199A388A341
:10270000E6EAF7E78591949120C08CE3F901808394
:102710001C828FEF8D8320E233E03F832E8324EDF4
:1027200033E03987288791E09BA79AA78C938CEA9E
:102730009DE09D8F8C8F8EED9DE09F8F8E8F84E727
:102740009EE099A388A38CE39FE09BA38AA3DF91DB
:10275000CF910895CF92DF92EF920F93CF93DF93B3
:10276000EC01FC01E158FF4F82E38083349781E064
:1027700090E0A0E0B0E080839183A283B3833B9795
:102780008FEF8083CE010E943B13CE010E941A1767
:102790006FEFCE010E941E176E018AE0C80ED11C99
:1027A000C6010E944508C6010E945508CE01489600
:1027B0000E9481178EE0E82E0FE020E14BE06DE0F3
:1027C000CE01825B9F4F0E94ED0CA596CE010E9428
:1027D000551465E0C6010E948208882351F060E02C
:1027E000CE01DF91CF910F91EF90DF90CF900C94BD
:1027F0000C1740E06EE473E0CE01DF91CF910F91B2
:10280000EF90DF90CF900C94F414CF93DF93D62FFA
:10281000C72F0E943113882359F0AD2FBC2FEBE84E
:10282000F7E784918D933196E53987E7F807C9F783
:10283000DF91CF91089550E0DA01AA0FBB1FA80FD6
:10284000B91F1F963C911F9750962C915097E32FDC
:10285000F22FE60FF11DE60FF11D259134919096B0
:102860003C932E935F97F90165917491FC017481FB
:10287000769F602D1124DC01A40FB51F91966C93F7
:102880009197F90185919491E92FF0E0862F90E0DE
:10289000E817F90720F4F90185919491692F769F43
:1028A000602D112492966C93089521E0FC012483FD
:1028B00024E020A72DEA33E0308B278740E060E05A
:1028C0000E941B1461E070E083E00E94BD18E1EB00
:1028D000F0E08081887F81608083F894109280008E
:1028E000E1E8F0E01082109285001092840088E107
:1028F00091E0909389008093880080818860808334
:10290000808181608083EFE6F0E080818260808357
:10291000789408950F93FC01842F01112AC062302E
:10292000D9F050F4662399F0613019F540E0682F32
:10293000CF010F910C941B146330A9F06430C9F4DB
:102940006481649F802D1124858F268F12C04B30A7
:1029500008F08AE0868B0DC06481649F802D11246D
:10296000818F228F06C06481649F802D1124838F04
:10297000248F0F910895FC0121110EC0648B848176
:10298000849F402D1124458B15A214A213A281E02F
:10299000878B80930304108E08958091030488230D
:1029A00019F08091000401C080E08093B400089584
:1029B000FC0161110DC0178A158A14A213A2108E92
:1029C0001092000410920104109203040C94CD1490
:1029D0000895CF93DF93611104C0EC010E94D814D5
:1029E0001982DF91CF9108950F931F93CF93DF93B7
:1029F000411110C08B01EC0160E00E94E9141E87B8
:102A00000D871B8A1A8A81E0898389E08E8B198E53
:102A10001B8E1D8EDF91CF911F910F910895CF9343
:102A2000DF93DC01611131C08C91882371F1119623
:102A30008C911197811129C019968C91199717962D
:102A40002C91179718969C911897E22FF92FE80F61
:102A5000F11DE80FF11D259134912F3F8FEF3807BD
:102A600011F41C9212C0ED013C873327220F331F53
:102A7000EA85FB85E20FF31F6591749140E0CD017B
:102A80000E94F41489858F5F8987DF91CF91089523
:102A900060E00C940F1560E00C94E9140F93CF9351
:102AA000DF93EC0161115CC08981882309F458C06F
:102AB0008D89811155C02D853E85EA89FB89EE0FF0
:102AC000FF1FE20FF31F85919491009701F589890B
:102AD000813021F41B8A1A8AF90110C01982888179
:102AE00060E0882371F0CE010E940F15EA89FB890E
:102AF000EE0FFF1F8D859E85E80FF91F859194913C
:102B000006C0CE01DF91CF910F910C94D814BC0177
:102B1000769567957695679580FF17C0AC0186E03E
:102B2000569547958A95E1F7292F2695269526955E
:102B300020514F716F7000E0CE010E948A14EA8923
:102B4000FB893196FB8BEA8BD3CF492F6F7320E043
:102B5000CE010E94BB148A899B8901969B8B8A8B2C
:102B6000DF91CF910F91089560E00C944E15CF93B3
:102B7000DF93EC016111BAC08F89882309F4B6C0D4
:102B80009D89911105C0CE01DF91CF910C94D8148D
:102B900091509D8B8DA1811139C02BA13CA12F5F3C
:102BA0003F4FC901880F991FEF8DF8A1E80FF91F5A
:102BB00065917491862F87708EA3AB0163E0569563
:102BC00047956A95E1F7CA0196958795972F96954F
:102BD00096959FA38F739C81899F802D11248DA32F
:102BE00041704093FF033CA32BA389A190E02817D9
:102BF000390760F02AA1222329F0821B91099CA3A6
:102C00008BA304C060E0CE010E94D8148DA1815036
:102C10008DA3888D21E0280F288F4C893FA1340F88
:102C20008C85380F3A836B8D662361F070E0822FBC
:102C3000022E000C990B0E94C31B8C8D869F300DB9
:102C400011243A838A8190E0CB966BE370E00E9476
:102C5000C31B8A833E893B83698D662371F0062EF0
:102C6000000C770B822F022E000C990B0E94C31BC5
:102C70008A8D869F300D11243B836D8D662389F0EC
:102C8000822F220F990B70E00E94C31BCB0162E0E0
:102C900070E00E94C31B2E8D9B81289F900D1124F4
:102CA0009B834F3341F08B818A300CF089E087FDA4
:102CB00080E08B8301C01B82F894EA81F0E0E45A43
:102CC000FC4FE491E09302048D8198A5899F802DAB
:102CD00011249B81899F802D11249EA1899F802D85
:102CE000112480930104809300047894DF91CF91A4
:102CF000089560E00C94B71560910104662329F1F2
:102D0000809104048F5F80930404909102048917DA
:102D1000E0F081E090910304911180E0809303043E
:102D2000109204048091FF03882369F080910001D0
:102D300093E4899F802D1124895B809300010E9478
:102D4000A31B909300040C94CD1408951F920F922E
:102D50000FB60F9211242F933F934F935F936F936E
:102D60007F938F939F93AF93BF93EF93FF930E94B3
:102D70007C16FF91EF91BF91AF919F918F917F91C1
:102D80006F915F914F913F912F910F900FBE0F90D8
:102D90001F901895CF93DF93EC0160E00E94E91437
:102DA00085EA93E09E878D871B8A1A8A81E0898352
:102DB00089E08E8B198E1B8E1D8EDF91CF91089529
:102DC000CF93DF93EC0160E00E94E9148DE993E07A
:102DD0009E878D871B8A1A8A81E0898389E08E8B82
:102DE000198E1B8E1D8EDF91CF910895CF93DF93A7
:102DF000EC0160E00E94E91487E993E09E878D87EB
:102E00001B8A1A8A81E0898389E08E8B198E1B8E3A
:102E10001D8EDF91CF910895FC01262F660F330B95
:102E20009681692F70E06F5F7F4FC9010E94C31BBD
:102E30008583089521E0FC012083089570E085E0FA
:102E40000C94BD18AF92BF92CF92DF92EF92FF9297
:102E50000F931F93CF93DF93EC0189819A812FE029
:102E6000289F8001299F100D112485E10E94A01840
:102E7000800F911F24E0969587952A95E1F79A8314
:102E800089832881222391F1EC81AD80B12CC12C62
:102E9000D12CA885B9857D0100E010E06E817F818D
:102EA0009B0140E050E08617970728F0BC01A81767
:102EB000B90708F4BD0180E090E01F921F921F92B5
:102EC000EF930E941E1B6B830F900F900F900F903B
:102ED00070E085E0DF91CF911F910F91FF90EF900F
:102EE000DF90CF90BF90AF900C94BD18DF91CF9141
:102EF0001F910F91FF90EF90DF90CF90BF90AF9018
:102F00000895FC018CE39FE09383828384E08183B6
:102F100081E084870895CF93DF93FC01248135817C
:102F2000232B79F1EC0184858F7141F584E10E94B6
:102F3000A018BC01990F880B990B0E94691C26EE02
:102F40003FE34EEC50E40E94F51C0E94381C9B01AC
:102F50007B836A83672B81F084E08983FE0134964A
:102F600080E0419151912417350710F4898309C0FD
:102F70008F5F8430B1F702C08FEF89838C858F5FBC
:102F80008C87DF91CF9108951F920F920FB60F9209
:102F900011242F933F938F939F93AF93BF9380916F
:102FA000060490910704A0910804B091090430919F
:102FB000050423E0230F2D3720F40196A11DB11D38
:102FC00005C026E8230F0296A11DB11D209305041C
:102FD0008093060490930704A0930804B093090417
:102FE00080910A0490910B04A0910C04B0910D04FF
:102FF0000196A11DB11D80930A0490930B04A09328
:103000000C04B0930D04BF91AF919F918F913F91AC
:103010002F910F900FBE0F901F9018952FB7F89417
:10302000609106047091070480910804909109044E
:103030002FBF08953FB7F89480910A0490910B0434
:10304000A0910C04B0910D0426B5A89B05C02F3F9C
:1030500019F00196A11DB11D3FBFBA2FA92F982FBE
:103060008827820F911DA11DB11DBC01CD0142E039
:10307000660F771F881F991F4A95D1F70895CF9241
:10308000DF92EF92FF92CF93DF936B017C010E945E
:103090001A18EB01C114D104E104F10479F00E9483
:1030A0001A186C1B7D0B683E7340A0F381E0C81AB0
:1030B000D108E108F108C851DC4FECCFDF91CF9186
:1030C000FF90EF90DF90CF900895789484B5826060
:1030D00084BD84B5816084BD85B5826085BD85B5BC
:1030E000816085BDEEE6F0E0808181608083E1E86B
:1030F000F0E01082808182608083808181608083A3
:10310000E0E8F0E0808181608083E1EBF0E08081A5
:1031100084608083E0EBF0E0808181608083EAE777
:10312000F0E0808184608083808182608083808100
:10313000816080838081806880831092C1000895BF
:103140008E3008F08E502091010190E4299F90016B
:1031500011248770822B80937C0080917A00806498
:1031600080937A0080917A0086FDFCCF8091780070
:103170002091790090E0922B08951F93CF93DF93D5
:10318000182FEB0161E00E944519209711F460E0CF
:1031900004C0CF3FD10539F461E0812FDF91CF9199
:1031A0001F910C948119E12FF0E0E754FC4FE4915A
:1031B000E330F9F048F4E130B9F0E230A1F584B53C
:1031C000806284BDC8BD34C0E630E9F0E73019F153
:1031D000E43049F580918000806280938000D09334
:1031E0008B00C0938A0024C084B5806884BDC7BDAD
:1031F0001FC080918000806880938000D0938900F8
:10320000C093880015C08091B00080688093B000A2
:10321000C093B3000DC08091B00080628093B00075
:10322000C093B40005C0C038D1050CF0B5CFAFCF06
:10323000DF91CF911F910895833081F028F4813080
:1032400099F08230A1F008958630A9F08730B9F066
:103250008430D1F4809180008F7D03C08091800004
:103260008F7780938000089584B58F7702C084B5EE
:103270008F7D84BD08958091B0008F7703C08091C9
:10328000B0008F7D8093B0000895CF93DF9390E0DE
:10329000FC01E353FC4F2491FC01EF51FC4F84915E
:1032A000882361F190E0880F991FFC01E75FFB4FD5
:1032B000C591D491FC01E150FC4FA591B4916111ED
:1032C00009C09FB7F8948881209582238883EC9168
:1032D0002E230BC0623061F49FB7F8948881322F9F
:1032E000309583238883EC912E2B2C939FBF06C0AF
:1032F0008FB7F894E8812E2B28838FBFDF91CF9171
:1033000008951F93CF93DF93282F30E0F901E754FE
:10331000FC4F8491F901E353FC4FD491F901EF5133
:10332000FC4FC491CC23C1F0162F81110E941C19AF
:10333000EC2FF0E0EE0FFF1FE150FC4FA591B49190
:103340009FB7F894111104C08C91D095D82302C076
:10335000EC91DE2BDC939FBFDF91CF911F910895FD
:10336000CF93DF93282F30E0F901E754FC4F84918D
:10337000F901E353FC4FD491F901EF51FC4FC49193
:10338000CC2391F081110E941C19EC2FF0E0EE0F7C
:10339000FF1FEB50FC4FA591B491EC91ED2381E020
:1033A00090E021F480E002C080E090E0DF91CF91D6
:1033B0000895CF92DF92EF92FF920F931F93CF93D6
:1033C000DF936C01EB017B01E40EF51E00E010E0E1
:1033D000CE15DF0561F06991D601ED91FC91019068
:1033E000F081E02DC6010995080F191FF1CFC80122
:1033F000DF91CF911F910F91FF90EF90DF90CF90D1
:1034000008956115710579F0FB0101900020E9F73D
:103410003197AF01461B570BDC01ED91FC91028007
:10342000F381E02D099480E090E00895EF92FF92FF
:103430000F931F93CF93DF937C01FB0100E010E01B
:103440006491EF012196662361F0D701ED91FC9123
:103450000190F081E02DC7010995080F191FFE01A9
:10346000EFCFC801DF91CF911F910F91FF90EF90A7
:103470000895DC01ED91FC910190F081E02D09941B
:103480000F931F93CF93DF93EC016DE00E94391AE5
:103490008C016AE0CE010E94391A800F911FDF91E2
:1034A000CF911F910F9108950F931F93CF93DF93A7
:1034B000EC010E94161A8C01CE010E94401A800F66
:1034C000911FDF91CF911F910F9108958F929F923D
:1034D000AF92BF92CF92DF92EF92FF920F931F9322
:1034E000CF93DF93CDB7DEB7A1970FB6F894DEBFC9
:1034F0000FBECDBF6C01142FE52FCB01022F19A2F7
:10350000223008F40AE07E0121E2E20EF11C802E56
:10351000912CA12CB12C612F7E2FA50194010E942A
:10352000D71B029F1019112481E0E81AF1081A3004
:1035300014F4105D01C0195CF7011083122FE32F02
:10354000CA01232B242B252B31F7B701C6010E947A
:10355000011AA1960FB6F894DEBF0FBECDBFDF9162
:10356000CF911F910F91FF90EF90DF90CF90BF9080
:10357000AF909F908F9008952115310541F4DC01A3
:10358000ED91FC910190F081E02D642F09940C9451
:10359000661A9A01AB0160E070E00C94BC1ACF92FD
:1035A000DF92EF92FF920F931F93CF93DF9321153A
:1035B000310581F4DC01ED91FC910190F081E02D69
:1035C000642FDF91CF911F910F91FF90EF90DF90CB
:1035D000CF9009942A30310501F577FF1DC06A01AB
:1035E0007B01EC016DE20E94391A8C0144275527BA
:1035F000BA014C195D096E097F092AE0CE010E94CB
:10360000661A800F911FDF91CF911F910F91FF904C
:10361000EF90DF90CF9008952AE0DF91CF911F9136
:103620000F91FF90EF90DF90CF900C94661A9A0163
:10363000AB01770F660B770B0C94CF1A4F925F920A
:103640006F927F92AF92BF92CF92DF92EF92FF92F2
:103650000F931F93CF93DF93CDB7DEB729013A01C4
:103660009B01AC01241935094609570989899A89B2
:10367000AB89BC89BC01CD016A197B098C099D0904
:103680000E94931BA801970124193509460957097F
:103690000E94F91BCA01B9016A0D7B1D8C1D9D1D7D
:1036A000DF91CF911F910F91FF90EF90DF90CF901E
:1036B000BF90AF907F906F905F904F900895089566
:1036C00061E08AE00E94811961E08AE00E94451968
:1036D0008CB580618CBD8CB580648CBD61E08DE063
:1036E0000E94451961E08BE00C944519811103C0DB
:1036F0008CB5806202C08CB58F7D8CBD08959CB561
:10370000937F892B8CBD08959CB59C7F282F2370B7
:10371000922B9CBD2DB582FB992790F9822F8E7F2D
:10372000892B8DBD0895DB018F939F930E94181CF8
:10373000BF91AF91A29F800D911DA39F900DB29F4D
:10374000900D11240895991B79E004C0991F9617D4
:1037500008F0961B881F7A95C9F780950895AA1BD3
:10376000BB1B51E107C0AA1FBB1FA617B70710F06C
:10377000A61BB70B881F991F5A95A9F7809590959E
:10378000BC01CD01089597FB072E16F4009407D0D5
:1037900077FD09D00E94AF1B07FC05D03EF4909541
:1037A00081959F4F0895709561957F4F0895A1E28F
:1037B0001A2EAA1BBB1BFD010DC0AA1FBB1FEE1FAB
:1037C000FF1FA217B307E407F50720F0A21BB30BF6
:1037D000E40BF50B661F771F881F991F1A9469F772
:1037E00060957095809590959B01AC01BD01CF01CE
:1037F0000895052E97FB1EF400940E94101C57FD9F
:1038000007D00E94D71B07FC03D04EF40C94101C69
:1038100050954095309521953F4F4F4F5F4F0895FC
:1038200090958095709561957F4F8F4F9F4F08952C
:103830000E94291CA59F900DB49F900DA49F800D00
:10384000911D11240895EE0FFF1F0590F491E02DB6
:103850000994A29FB001B39FC001A39F700D811D69
:103860001124911DB29F700D811D1124911D089589
:103870000E94D41C88F09F5798F0B92F9927B75110
:10388000B0F0E1F0660F771F881F991F1AF0BA9504
:10389000C9F714C0B13091F00E94EE1CB1E0089558
:1038A0000C94EE1C672F782F8827B85F39F0B93F4A
:1038B000CCF3869577956795B395D9F73EF49095B7
:1038C0008095709561957F4F8F4F9F4F0895E89435
:1038D00009C097FB3EF490958095709561957F4F58
:1038E0008F4F9F4F9923A9F0F92F96E9BB27939506
:1038F000F695879577956795B795F111F8CFFAF416
:10390000BB0F11F460FF1BC06F5F7F4F8F4F9F4F46
:1039100016C0882311F096E911C0772321F09EE8A4
:10392000872F762F05C0662371F096E8862F70E00A
:1039300060E02AF09A95660F771F881FDAF7880FE4
:103940009695879597F9089597F99F6780E870E0B5
:1039500060E008959FEF80EC089500240A94161605
:10396000170618060906089500240A94121613066D
:10397000140605060895092E0394000C11F48823FB
:1039800052F0BB0F40F4BF2B11F460FF04C06F5F17
:103990007F4F8F4F9F4F089557FD9058440F551FED
:1039A00059F05F3F71F04795880F97FB991F61F0C1
:1039B0009F3F79F087950895121613061406551F38
:1039C000F2CF4695F1DF08C0161617061806991FA4
:1039D000F1CF86957105610508940895E894BB2799
:1039E00066277727CB0197F908950E94081D0C944C
:1039F000BB1C0E94AD1C38F00E94B41C20F0952323
:103A000011F00C94A41C0C94AA1C11240C94EF1C0F
:103A10000E94CC1C70F3959FC1F3950F50E0551F89
:103A2000629FF001729FBB27F00DB11D639FAA2713
:103A3000F00DB11DAA1F649F6627B00DA11D661F62
:103A4000829F2227B00DA11D621F739FB00DA11D83
:103A5000621F839FA00D611D221F749F3327A00D3D
:103A6000611D231F849F600D211D822F762F6A2FD9
:103A700011249F5750409AF0F1F088234AF0EE0F3E
:103A8000FF1FBB1F661F771F881F91505040A9F76B
:103A90009E3F510580F00C94A41C0C94EF1C5F3FDA
:103AA000E4F3983ED4F3869577956795B795F795A7
:103AB000E7959F5FC1F7FE2B880F911D969587951F
:103AC00097F90895DC0101C06D9341505040E0F733
:103AD0000895FB01DC014150504048F001900D92E7
:103AE0000020C9F701C01D9241505040E0F70895F1
:043AF000F894FFCF78
:103AF4000101001923000000008602000000005F9D
:103B04001B00000000000000000000000000000096
:103B140000D7060000EC060000000000005B040073
:103B2400009E0400007C040000BF040000000000AC
:103B34000000000000000000000000000000000081
:103B44000000000000000000005C0700002D0700DA
:103B5400000000000000000000520ED9194C4F4133
:043B64004445520082
:040000030000046A8B
:00000001FF
